:100000000C94A4020C94C1020C94C1020C94C10281
:100010000C94C1020C94C1020C94C1020C94C10254
:100020000C94C1020C94C1020C94C1020C941E03E6
:100030000C9498030C94C1020C94C1020C94C1025C
:100040000C94C1020C94C1020C9407050C94C102DB
:100050000C94C1020C94C1020C94C1020C94C10214
:100060000C94C1020C94C1020000000000000000CA
:100070000000000000096000000000000071310075
:1000800000007A736177320000637864653433006E
:100090000020766674723500006E626867793600FB
:1000A00000006D6A75373800002C6B696F303900BD
:1000B000002E2F6C3B702D00000027005B3D0000E0
:1000C00000000A5D005C0000000000000000080065
:1000D0000031003437000000302E323536381B0036
:1000E000002B332D2A390000000000000000000022
:1000F0000000000000097E00000000000051210007
:1001000000005A53415740000043584445242300FF
:100110000020564654522500004E424847595E0082
:1001200000004D4A55262A00003C4B494F29280023
:10013000003E3F4C3A505F00000022007B2B000045
:1001400000000A7D003F00000000000000000000E9
:10015000000000000000000000000000000000009F
:10016000000000000000000000000000000000008F
:10017000000000000000000000000000000000007F
:10018000000000000000000000000000000000006F
:10019000000000000000000000000000000000005F
:1001A000000000000000000000000000000000004F
:1001B000000000000000000000000000000000003F
:1001C000000000000000000000000000000000002F
:1001D000000000000000000000000000000000001F
:1001E000000000000000000000000000000000000F
:1001F00000000000000000000000000000000000FF
:1002000000000000000000000000000000000000EE
:1002100000000000000000000000000000000000DE
:1002200000000000000000000000000000000000CE
:1002300000000000000000000000000000000000BE
:1002400000000000000000000000000000000000AE
:1002500010101010100010002828000000000000EE
:100260002828FE28FE28280010781438503C10005A
:10027000004C2C10686400001814081462225C0002
:1002800010100000000000002010080808102000D6
:1002900008102020201008001092543854921000AA
:1002A000101010FE10101000000000003030201060
:1002B000000000FE000000000000000000303000E0
:1002C000804020100804020038444454444438005C
:1002D00010181010101038003844402010087C000E
:1002E00038444030404438003028247C20207000BE
:1002F0007C04043C404438003844043C4444380006
:100300007C40201008080800384444384444380031
:100310003844447840443800003030003030000029
:100320000030300030302010201008040810200069
:100330000000FE00FE000000040810201008040069
:1003400038444020100010003844745474043800BD
:100350003844447C444444003C44443C44443C00D1
:1003600038440404044438003C44444444443C00BD
:100370007C04043C04047C007C04047C040404002D
:1003800038440474444438004444447C44444400A5
:10039000381010101010380070202020242418006D
:1003A0004444241C24444400080808080808780031
:1003B00082C6AA9282828200444C5454644444000F
:1003C0003844444444443800384848380808080051
:1003D00038444444444438603C44443C142444007D
:1003E00038440438404438007C10101010101000BD
:1003F00044444444444438004444442828101000F1
:1004000082828254542828004444281028444400FE
:1004100044442810101010007C40201008047C0078
:100420003808080808083800020408102040800036
:100430003820202020203800102844000000000030
:1004400000000000000000FE081000000000000096
:10045000003840784444B800080838484848340018
:100460000000380404043800404070484848B00098
:10047000000038447C0438003048081C0808080094
:100480000000B844447840380404344C44444400E8
:100490000010001010101000001000101010100CB0
:1004A000040424140C142400181010101010100050
:1004B00000006D9292828200000034484848480053
:1004C00000003844444438000000344848380808E4
:1004D00000005824243820200000340C04040400B8
:1004E0000000380418201C000010381010101000F4
:1004F0000000242424245800000044444428100010
:100500000000828292AA440000004428102844007F
:10051000000048484870403800003C2010083C006B
:1005200030080804080830001010101010101000D7
:100530000C10102010100C0000000C926000000045
:10054000000000000000000011241FBECFEFD4E027
:10055000DEBFCDBF11E0A0E0B1E0ECE6F1E102C00A
:1005600005900D92AE32B107D9F712E0AEE2B1E0DC
:1005700001C01D92A538B107E1F70E9406030C9453
:10058000B4080C9400004423D1F1813621F4809109
:100590002F01816029C0833721F480912F0182606F
:1005A00023C0843621F480912F0184601DC08636DB
:1005B00021F480912F01886017C08A3621F4809140
:1005C0002F01806111C08B3621F480912F01806250
:1005D0000BC08C3621F480912F01806405C08B33D1
:1005E00031F480912F01806880932F0108958B3121
:1005F00031F410926A0110926B0110922D0108954E
:10060000E1E6F0E080E8808310820895F8948DEFB1
:1006100084B98FE78AB90E9402040E94E5030E9410
:1006200000030E9475050E94FE06789483B78160DE
:1006300083BF889583B78E7F83BFF8CF1F920F92B9
:100640000FB60F9211248F939F9318B880913201A7
:100650008823B9F18F5F80933201823031F482E4D4
:1006600090E090938B0080938A00809132018830D3
:1006700019F486E093E004C08E3039F480E490E011
:1006800090938B0080938A004CC0833129F4809131
:10069000310180FF46C006C0843169F48091310188
:1006A00080FD3FC087E297E09093890080938800A7
:1006B0008EE790E0E5CF8E31A1F51092320181E016
:1006C0002EC080913001823F49F58091310180FF39
:1006D0000EC082E0809332011092300183E993E0F2
:1006E000909389008093880082E490E00DC081E0BF
:1006F000809332011092300183E993E09093890056
:10070000809388008EE790E090938B0080938A001E
:10071000809131018F5F8093310103C08F5F80939F
:1007200030019F918F910F900FBE0F901F901895E1
:100730001F920F920FB60F9211242F933F934F9356
:100740005F936F937F938F939F93AF93BF93EF9339
:10075000FF9385E088B989E08A95F1F700C0539A44
:100760008AE05B9A5B9800008150D9F7539885E046
:1007700088B983E18A95F1F70000809132018823DE
:1007800051F0843110F480FF0FC08091350188BD95
:1007900088B587BD07C08091350188BD88B587BD04
:1007A0000E94A6050E94D406FF91EF91BF91AF91E0
:1007B0009F918F917F916F915F914F913F912F9179
:1007C0000F900FBE0F901F9018952FE027B9539AE6
:1007D000109285001092840088E297E0909389003F
:1007E0008093880084EF91E090938B0080938A003F
:1007F0001092800089E08093810086E080936F00F2
:1008000028B908958AB180668AB981EA84BD81E0F9
:1008100085BD16BC81EE9CEA909341018093400116
:10082000909338018093370190933F0180933E016C
:1008300090933D0180933C01089560913A01862F89
:1008400090E09C012F71307021153105A9F4409181
:100850004001509141019A012170307030952195ED
:100860003F4F2070347B569547952427352730938A
:1008700041012093400150C09C012F703070213005
:100880003105A9F440913701509138019A01217046
:100890003070309521953F4F2070347B56954795A9
:1008A00024273527309338012093370135C09C0128
:1008B0002770307022303105A9F440913E015091EB
:1008C0003F019A0121703070309521953F4F207083
:1008D000347B569547952427352730933F01209345
:1008E0003E011AC09C012370307023303105A1F401
:1008F00040913C0150913D019A012170307030953A
:1009000021953F4F2070347B5695479524273527F6
:1009100030933D0120933C0183709070009731F437
:10092000809139018C5F8093390117C08130910526
:1009300031F4809133018B5F809333010EC082309C
:10094000910531F4809134018A5F8093340105C0B0
:1009500080913B01885F80933B016F5F60933A0118
:100960001092350130913601832F30FF05C09091F0
:1009700040019F739093350181FF08C0209137019A
:100980002F7390913501920F9093350182FF08C02B
:1009900020913E012F7390913501920F9093350174
:1009A00083FF08C020913C012F7390913501920F75
:1009B0009093350184FF09C0209139012695269531
:1009C00090913501920F9093350185FF09C02091D8
:1009D00033012695269590913501920F909335011C
:1009E00086FF09C0909134019695969580913501C6
:1009F000890F8093350137FF09C090913B0196958F
:100A0000969580913501890F8093350108951F9245
:100A10000F920FB60F9211242F933F934F935F9332
:100A20006F937F938F939F93AF93BF93EF93FF93B6
:100A30006091C600603F21F480912E01816042C028
:100A4000603E21F480912E0182603CC06F37B8F582
:100A500080912E0181FD33C0623119F06935C1F4F6
:100A600006C080FF02C0877F07C0886005C080FF86
:100A700002C08B7F01C0846080932E0180912E0183
:100A8000982F9C7011F0806101C08F7E80932E01A1
:100A900090912E0194FF09C06E3038F0603628F432
:100AA000E62FF0E0E851FF4F04C0E62FF0E0E859F0
:100AB000FF4F849141E090FD40E00E94C30280918D
:100AC0002E018C7F80932E01FF91EF91BF91AF910A
:100AD0009F918F917F916F915F914F913F912F9156
:100AE0000F900FBE0F901F9018958AB18C7E8AB917
:100AF0008BB180718BB980E98093C10086E78093C8
:100B0000C2000895539AA82FB92F70E095E08FE0A6
:100B100018C0FF27E7FDF09523E0EE0FFF1F2A9591
:100B2000E1F7E60FF71FE85BFE4FE49129E0E0FFF5
:100B300002C088B902C098B90000215011F0E695B2
:100B4000F6CFED91EE2329F7539808956091300187
:100B5000603158F480912D01873008F024C1862F30
:100B600090E001970E9450070895603240F5669525
:100B7000677080E091E00E94820589E08A95F1F734
:100B800000C0609130016695677082E892E00E9433
:100B9000820590E39A95F1F7609130016695677050
:100BA00083E091E00E948205A9E0AA95F1F700C0D8
:100BB00060913001669567708CE692E046C0809146
:100BC0002D01633298F4882339F0833029F08A307C
:100BD00019F08B3009F0E7C0B3E4BA95F1F78FE074
:100BE00088B988EC90E00197F1F7A7C0883008F445
:100BF00042C010923601962F90549032E8F493E15F
:100C00009A95F1F70000883031F466956695677023
:100C100086E091E01AC0893031F466956695677078
:100C20008FE091E012C08A3009F0BDC066956695EC
:100C3000677088E191E009C0862F8056803240F4C9
:100C400066956695677082E291E00E94820508953C
:100C5000A8E1AA95F1F789E088B98EE00000539ADF
:100C600099E05B9A00005B989150D9F70000539887
:100C70008150A1F763C0653C08F04BC090917702AA
:100C800080FF03C085E088B903C089E088B900000F
:100C9000BEE3BA95F1F7000000000000000000007C
:100CA00000000000000088E035E049E0000000009E
:100CB00000000000000000000000000090FF03C0E2
:100CC00048B9539A04C038B900000000000029E078
:100CD0005B9A00005B982150D9F753980000000000
:100CE000000000000000000038B9815011F0969516
:100CF000DDCF80912D0180FF02C089E001C085E039
:100D000088B980913001843C09F44DC00E940107EC
:100D10000895683CB0F4982F9150923028F08430B8
:100D200019F0853009F03FC083E48A95F1F78FE030
:100D300088B9A8ECB0E01197F1F7000085E088B918
:100D40000895603E50F5B4E4BA95F1F7E8E7F2E0B3
:100D500020EE30E065E079E0819190E0880F991F06
:100D6000880F991F40913001D901A41BB1098A173E
:100D70009B0714F078B902C068B90000539A89E063
:100D80005B9A00005B988150D9F70000539868B9CE
:100D9000B2E0E038FB0701F70895862F90E0805F0E
:100DA00090400E94500708950E941D040895E2E6B5
:100DB000F1E0AFE6B2E0819181508D9381E0EA36B7
:100DC000F807C9F710927702089510926201109205
:100DD00063011092640110926501109266011092F5
:100DE000670110926801109269010895E2E4F1E050
:100DF000119281E0E236F807D9F708950E94E506DE
:100E00000895FF920F931F9380912D01882311F075
:100E1000833029F42091300180E290E004C02091D9
:100E2000300188EC90E0821B91099595879520917F
:100E3000800230918102820F931FEFE6F2E020E002
:100E400030E000E011E0F0804F2D4F3FD9F06F2DE2
:100E500070E0DB01A459BE4FA20FB31F4C9150E0CC
:100E6000481759077CF06E5B7E4FDB016C91612364
:100E700029F448505040841795071CF4FA94F082E6
:100E800001C0012B110F3196205E3F4FB1E02030A1
:100E90003B07C9F6009377021F910F91FF900895C9
:100EA0008930910509F4BDC08A30910534F497FD6D
:100EB00041C18830910574F0A6C08B30910509F4CA
:100EC00028C18B3091050CF4BAC08C30910509F023
:100ED00031C122C121E030E0082E02C0220F331FB1
:100EE0000A94E2F7FC01E858FD4F3081332319F0F2
:100EF0003150308307C0422F409530913601342362
:100F000030933601FC01E858FD4F3081332309F05E
:100F100011C140912F01322F342309F40BC1322F1C
:100F20003095342330932F014091800250918102FB
:100F3000BA01615070406E3F710508F0FBC03091FE
:100F40002D01332311F0333091F4DC01AE59BE4F43
:100F50003C91FC0155E0EE0FFF1F5A95E1F7E30FBE
:100F6000F11DE459FE4F40833F5F3C932AC0FC01D2
:100F7000E159FD4FE081EF3F09F4DCC04091770279
:100F8000422361F0F0E0EE5BFE4F4081542F52238C
:100F900029F4422B4083313021F405C03130E1F493
:100FA0001DC0353029F440916B014E5F40936B01B9
:100FB000323011F0343029F430916A013E5F3093C1
:100FC0006A0188589D4F38E0FC01308380913601DA
:100FD000822B809336010895353039F480916B016E
:100FE00018161CF4815080936B01323019F03430A4
:100FF00009F0A0C080916A0118160CF09BC08150C6
:1010000080936A01089580916A016AE00E949B08BA
:10101000805D80938202905D90938302109284029F
:10102000089580916B016AE00E949B08805D809327
:101030006C02905D90936D0210926E020895809103
:1010400080029091810201969093810280938002A8
:10105000F1E080309F0709F059C020912D01222333
:10106000C1F12630B1F1E2E6F1E041E030E00CC040
:101070005D91542309F43F5FA817B907C9F781E0D0
:10108000EA36F80741F0440F8191A2E4B1E090E024
:101090008A0F9B1FF1CF213011F0253029F4809168
:1010A0006B01831B80936B01223011F0243029F4F3
:1010B00080916A01831B80936A0180916B0187FF95
:1010C00002C010926B0180916A0187FF02C01092EA
:1010D0006A0180E89FEF9093810280938002809163
:1010E0002D018F5F80932D01863011F410922D0118
:1010F00080912D01882311F0833031F40E94E506A0
:1011000010928102109280020E94F60610927702DD
:1011100008950E94D706089580916A0184361CF0D4
:1011200088E080932D0180916B0184361CF089E06A
:1011300080932D01089587FB082E062687FD819553
:1011400067FD619505D00EF4919507FC8195089592
:10115000991B79E004C0991F961708F0961B881F09
:0C1160007A95C9F780950895F894FFCFA8
:10116C005031005032002050312057696E730020EE
:10117C0050322057696E73005249464652494445D5
:0E118C00520050726573732065736321000A70
:00000001FF
